:020000040000FA
:020000000428D2
:040002000034003492
:080008008C0123008C01210092
:100010006A30990021000F308C0022009D141D14BD
:1000200025000F309300250091012000FF309B0038
:10003000200001309C0020008B010C168C16AF01B3
:100040002000A201A301A401A501A601A701A0010E
:10005000A10164000C193D280C193F280030200232
:1000600003192A280730200203184328A10A0C305C
:10007000210203194628A0012A28000000000000E0
:100080006400A00A2A28A001A1012A28A001A10138
:100090000C1956280C19582800302002031948283A
:1000A0000730200203185C28A00148280000000047
:1000B00000006400A00A482896019701A001A10150
:1000C000A1150C1974280C19762800302002031988
:1000D00061280730200203187A28A20D2214A10BF0
:1000E00072287E28A0016128000000000000640042
:1000F000A00A6128A20D2210A10B7228A001A10163
:100100000C198E280C199028003020020319802821
:100110000730200203189428A001202800000000C6
:1001200000006400A00A8028A001A101A1150C19FB
:10013000AA280C19AC280030200203199728073090
:1001400020020318B028A30D2314A10BA828B4285B
:10015000A00197280000000000006400A00A972872
:10016000A30D2310A10BA828A001A1010C19C428DC
:100170000C19C628003020020319B62807302002C7
:100180000318CA28A0012028000000000000640015
:10019000A00AB628A001A101A1150C19E0280C198C
:1001A000E228003020020319CD280730200203186E
:1001B000E628A40D2414A10BDE28EA28A001CD28EE
:1001C0000000000000006400A00ACD28A40D241047
:1001D000A10BDE28A001A1010C19FA280C19FC289A
:1001E000003020020319EC280730200203180029F0
:1001F000A0018C290000000000006400A00AEC2887
:10020000A001A101A1150C1916290C1918290030FB
:100210002002031903290730200203181C29A50D09
:100220002514A10B14292029A00103290000000096
:1002300000006400A00A0329A50D2510A10B1429B4
:10024000A001A1010C1930290C193229003020021B
:10025000031922290730200203183629A0018C290E
:100260000000000000006400A00A2229A001A101F2
:10027000A1150C194C290C194E2900302002031924
:1002800039290730200203185229A60D2614A10B84
:100290004A295629A0013929000000000000640005
:1002A000A00A3929A60D2610A10B4A29A001A101F7
:1002B0000C1966290C1968290030200203195829E5
:1002C0000730200203186C29A0018C2900000000CF
:1002D00000006400A00A5829A001A101A1150C1971
:1002E00082290C1984290030200203196F29073054
:1002F000200203188829A70D2714A10B80298C2917
:10030000A0016F290000000000006400A00A6F290E
:10031000A70D2710A10B80296400220823062406BC
:10032000250626062706031D20280030AE22A90038
:100330000130AE22AA000330AE22AB000530AE225F
:10034000AC002308FE39A80020001C15200022085C
:100350002906031DE62928082A06031DE62964004C
:10036000192364002318CD296400292300006400A8
:10037000250016100000961400008C1600002000C6
:100380002C082500910020002B1C20286400092344
:10039000640025009101200020286400292300002A
:1003A0006400250096100000161400000C160000D2
:1003B00020002C082500910020002B1C2028640020
:1003C0000923640025009101200020282209031D33
:1003D000EB29AF01202822080319972AA21BF6292E
:1003E0007039703A0319052AAF012028AF0120287F
:1003F000EC302302031D2028073024060319B92AF4
:100400002508B10024089D221D282F1CF429A508C9
:1004100003194F2A2208783A0319172A2208743A36
:100420000319352A22087C3A03193D2A2028241A68
:1004300020282308AE22B0002822B005A41D242ABB
:100440003008031DE022202830080319E02220286C
:1004500001308A0024080739820701340234043449
:10046000083410342034403480342308AE2224026F
:10047000031D2028AF01E022202807302306031D9A
:10048000462A08302406031DDD2ABD2A2408B100AF
:1004900023089D22AF016400E02264002028221D71
:1004A000612AA2182028221C802A562A2308AD007F
:1004B000AD030310AD0D0310AD0DAF146400E022C9
:1004C0002028AF1C2028220803392D07AE00073052
:1004D0002E060319B42AA21D762A2308B1002E087D
:1004E0009D22AE01AF016400E02220282E08AE223A
:1004F0002302031D2028AE01AF016400E022202862
:10050000AF1C2028A21D8D2A2308B1001C309D227B
:10051000AD01AF016400E02220281C30AE2223028E
:10052000031D2028AD01AF016400E022202822082D
:100530002306031D20282F14202864002300910087
:100540002000310823009300151555309600AA307D
:10055000960095149518AA2A2000080023009100FF
:10056000151413082000080008302306031DDD2A97
:10057000BD2A08302506031D20288130B100003037
:100580009D22F830B10001309D220530B1000230CB
:100590009D220130B10003309D220130B1000430B2
:1005A0009D227F30B10005309D225E30B1000630C3
:1005B0009D229C30B10007309D22AD012F101D28D7
:1005C0006400250016100000961400008C16000030
:1005D00020000F302500910020006400002300233C
:1005E0000023002300230023640025009101200044
:1005F0000800000064000230B200B20BFD2A0800BF
:100600004730B300F922042BB30B022B0000640027
:1006100008000230AE22B7000A30B500C830B6007C
:1006200000006400B60B102BB50B0E2BB70B0C2B78
:1006300008000430AE22B7000A30B500C830B6005A
:1006400000006400B60B202BB50B1E2BB70B1C2B28
:1006500008001430B60000006400B60B2B2B080015
:020000040001F9
:02000E009C0F45
:02001000FF3AB5
:10E000008100F8000500010001007F005E009C0017
:00000001FF
